:020000040000FA
:100000002500050483061C0A58071D0A17020E0E58
:1000100037000600C80C02005804B409010CB000F7
:100020000307B10030024307190A31024307190AD6
:100030000008580506020300E209090C24006000CC
:10004000A40204021F0E43071F0A660076000E0C6E
:1000500037000600C80C020072007300E209A6090E
:10006000310AD1092607310A4607310A72007300A6
:10007000D10926073E0A4607420A360A4607310AD0
:100080007805460A2607310A7804460AD109780716
:100090004E0A2606360A4606460A530A4606360A17
:1000A0002606460A530AD109B2024306B3022607BE
:1000B000530A4607530A050C3500D109B20243061C
:1000C000B302430603007807680A26065B0A6B0A38
:1000D00046065B0A6B0AF5025D0AD109B2024306C5
:1000E000B3024306030078077A0A26060300460691
:1000F0006D0A7F0A4606030026066D0A7F0AD109AB
:1001000026077F0A46077F0A330243078E0A1A0C26
:10011000920003068E0A050C3200920A140CB200FB
:100120000307F300A6093805D70938049C09E2093A
:10013000AD09DE09A609930A7807A10A3604370437
:10014000A30A560457041702060000083605560590
:100150003705570517020600000836045604370411
:1001600057041702060000083807C20A0602960163
:1001700057017807BD0A020EBE0A040E4306C20AE2
:100180001805C60A050C34001804C60A1807CB0A5D
:10019000F4004306CC0A00080E0C37000600580491
:1001A0000300010C30007100580506020300120222
:1001B000300013023100580506020300CA0C020089
:1001C0000400E60ACC0C02000400E60A010C300030
:0801D00071005805060203004E
:021FFE00EF0FE3
:00000001FF
